:02000000542F7B
:100006006400031C0C288312031305148514851041
:0E0016001128831203130510851485100800AD
:100024008316031398181828000012282608831230
:040034009900080027
:0E0038000030831203138C1A0130F000080010
:1000460064008312031305158615B4013408073CB2
:10005600031C3228EC0CEC130320B40A29280511E2
:10006600B40134080F3C031C432808303402031C37
:100076003D280515EA0CE90CEA130320B40A3428D6
:10008600B4013408073C031C4D28EB0CEB1303208A
:10009600B40A4428B4013408073C031C5728E40D6D
:1000A60064100320B40A4E2805110D30FD00FD0B27
:0800B6005A2805158615080003
:1000BE00831203131A08E300981C672818121816E7
:0600CE006308F0000800C9
:1000D400831603139816903083129800831686149F
:1000E400061183128C1E79281A08F0007328080060
:1000F40083160313A50183126F0884000008831676
:10010400A4002408003A031994282408A600122005
:100114008316A50A250883126F0784000008831636
:06012400A400832808007E
:10012A0083120313FB01FA01F901F801A001730D0F
:10013A00F80D7408F8027508031C750FF9027608A1
:10014A00031C760FFA027708031C770FFB020001E3
:10015A00031C0130A002F30D0730FC00730DF80DEB
:10016A00F90DFA0DFB0DA00D7408731CCE28F802C8
:10017A007508031C750FF9027608031C760FFA023C
:10018A007708031C770FFB020001031C0130A00251
:10019A00DF28F80775080318750FF907760803189A
:1001AA00760FFA0777080318770FFB070001031881
:1001BA000130A007F30DFC0BB328720DF80DF90DF1
:1001CA00FA0DFB0DA00D7408731CFD28F8027508C2
:1001DA00031C750FF9027608031C760FFA027708DA
:1001EA00031C770FFB020001031C0130A0020E2939
:1001FA00F80775080318750FF90776080318760FBC
:10020A00FA0777080318770FFB0700010318013074
:10021A00A007F20D0730FC00720DF80DF90DFA0D6A
:10022A00FB0DA00D7408721C2C29F8027508031C1A
:10023A00750FF9027608031C760FFA027708031C79
:10024A00770FFB020001031C0130A0023D29F807C9
:10025A0075080318750FF90776080318760FFA0759
:10026A0077080318770FFB07000103180130A0076E
:10027A00F20DFC0B1129710DF80DF90DFA0DFB0D9C
:10028A00A00D7408721C5B29F8027508031C750F0F
:10029A00F9027608031C760FFA027708031C770F17
:1002AA00FB020001031C0130A0026C29F807750843
:1002BA000318750FF90776080318760FFA077708F7
:1002CA000318770FFB07000103180130A007F10D8F
:1002DA000730FC00710DF80DF90DFA0DFB0DA00D9C
:1002EA007408711C8A29F8027508031C750FF90233
:1002FA007608031C760FFA027708031C770FFB02B5
:10030A000001031C0130A0029B29F8077508031895
:10031A00750FF90776080318760FFA077708031896
:10032A00770FFB07000103180130A007F10DFC0B42
:10033A006F29700DF80DF90DFA0DFB0DA00D74085B
:10034A00711CB929F8027508031C750FF9027608A1
:10035A00031C760FFA027708031C770FFB020001D1
:10036A00031C0130A002CA29F80775080318750F83
:10037A00F90776080318760FFA0777080318770F34
:10038A00FB07000103180130A007F00D0730FC003D
:10039A00700DF80DF90DFA0DFB0DA00D7408701C07
:1003AA00E829F8027508031C750FF9027608031C80
:1003BA00760FFA027708031C770FFB020001031C71
:1003CA000130A002F929F80775080318750FF90713
:1003DA0076080318760FFA0777080318770FFB07D2
:1003EA00000103180130A007F00DFC0BCD2970188D
:1003FA000C2A7408F80775080318750FF9077608A8
:10040A000318760FFA0777080318770FFB07080017
:10041A001C2070080319152A5F207008DA00162AB2
:04042A000D2A08008F
:10042E00293083120313EC009B30E900B230EA004E
:10043E001030EB00E40123202830EC00B030E9004E
:10044E001630EA00AA30EB00E401232006168612CD
:06045E00061386130800DE
:0E046400831203136E088A006D0882000800E0
:10047200831203137008F100F0010830FC007108C8
:10048200F40C0318482AFC0B412AF1010034031032
:100492004D2AF40C0318F107F10CF00CFC0B4A2A5C
:0204A200080050
:1004A400831203132230FC00F801F901FA01FB0165
:1004B400FC030319882A0310FB0CFA0CF90CF80C42
:1004C400F30CF20CF10CF00C031C5A2AFC03031974
:1004D4007A2A7408F80775080318750FF90776085F
:1004E4000318760FFA0777080318770FFB075E2ABD
:1004F4007408F80775080318750FF90776080318C8
:0E050400760FFA0777080318770FFB07080039
:100512006400831203133508F0000A30F400392214
:100522007008D5007108D6000030D61BFF30D70006
:10053200D8000130B400073034020318C62A340848
:10054200353E84000008F000F101F201F301550884
:10055200F00756080318560FF10757080318570FEC
:10056200F20758080318580FF3070A30F400F50190
:10057200F601F70152227008D5007108D600720800
:10058200D7007308D800B40A9C2A3C08F000F10195
:10059200F201F3015508F00756080318560FF10748
:1005A20057080318570FF20758080318580FF30794
:1005B2007008D5007108D6007208D7007308D800F9
:0205C20008002F
:1005C400293083120313EC005908003EE900B230CD
:1005D4000318013EEA001030EB00232005118514B6
:1005E400051086110630FD00FD0BF62A00002830A8
:1005F400EC003108E9003208EA00AA30EB002320BD
:1006040005118514051086115508DF005608E00011
:0A0614005708E1005808E200080052
:10061E000030831203135802031D1F2B153057028F
:10062E00031D1F2B35305602031D1F2BAF305502F5
:10063E000318322B5808013C031D2F2B5708D93CA9
:10064E00031D2F2B5608053C031D2F2B5508C03CB0
:10065E000318322B0F2B01305802031D402B8C3008
:10066E005702031D402B93305602031D402B703052
:10067E005502031C5F2B5808013C031D502B5708D5
:10068E00D83C031D502B5608DE3C031D502B55083D
:10069E00B03C031C5F2BFF30D900061286120613E6
:1006AE0086170430AF007230AD000630AE00212D3B
:1006BE0001305802031D6D2B5E305702031D6D2B4A
:1006CE00CC305602031D6D2BB0305502031C8C2B03
:1006DE005808013C031D7D2B57088C3C031D7D2BB8
:1006EE005608933C031D7D2B55086F3C031C8C2B29
:1006FE00FF30D90006168616061786130430AF0093
:10070E00FB30AD000430AE00212D01305802031D28
:10071E009A2B31305702031D9A2B05305602031DBA
:10072E009A2BF0305502031CB92B5808013C031DBF
:10073E00AA2B57085E3C031DAA2B5608CC3C031D62
:10074E00AA2B5508AF3C031CB92BF730D900061263
:10075E008616061786130430AF00D430AD00033072
:10076E00AE00212D01305802031DC72B0A3057024F
:10077E00031DC72BE0305602031DC72B5030550208
:10078E00031CE62B5808013C031DD72B5708313CA0
:10079E00031DD72B5608053C031DD72B5508EF3CE0
:1007AE00031CE62BF730D9000616861206178613A1
:1007BE000430AF000330AD000330AE00212D003009
:1007CE005802031DF42BB6305702031DF42BF330E1
:1007DE005602031DF42BF0305502031C132C58083F
:1007EE00013C031D042C57080A3C031D042C56081B
:1007FE00E03C031D042C55084F3C031C132CFB300E
:10080E00D90006128612061786130430AF002E305A
:10081E00AD000230AE00212D00305802031D212CF8
:10082E0089305702031D212C2D305602031D212C19
:10083E0030305502031C402C5808003C031D312C4F
:10084E005708B63C031D312C5608F33C031D312CC2
:10085E005508EF3C031C402CF330D90006168616C3
:10086E00061386130430AF008830AD000130AE00A1
:10087E00212D00305802031D4E2C5B305702031DF4
:10088E004E2C66305602031D4E2C70305502031C42
:10089E006D2C5808003C031D5E2C5708893C031D27
:1008AE005E2C56082D3C031D5E2C55082F3C031C58
:1008BE006D2CDB30D900061286160613861308300F
:1008CE00AF003830AD000230AE00212D003058029E
:1008DE00031D7B2C44305702031D7B2CAA3056027D
:1008EE00031D7B2C20305502031C9A2C5808003C0B
:1008FE00031D8B2C57085B3C031D8B2C5608663C46
:10090E00031D8B2C55086F3C031C9A2CD330D90039
:10091E0006128616061386130830AF008830AD0017
:10092E000130AE00212D00305802031DA82C2D30B1
:10093E005702031DA82CC6305602031DA82CC0302A
:10094E005502031CC72C5808003C031DB82C570831
:10095E00443C031DB82C5608833C031DB82C550887
:10096E000F3C031CC72C9B30D900061686120613AB
:10097E0086131030AF003F30AD000230AE00212D97
:10098E0000305802031DD52C21305702031DD52CE3
:10099E0091305602031DD52CC0305502031CF42C89
:1009AE005808003C031DE52C57082D3C031DE52C73
:1009BE0056089F3C031DE52C5508AF3C031CF42C38
:1009CE009330D90006168612061386131030AF0028
:1009DE00C730AD000130AE00212D00305802031D8E
:1009EE00022D15305702031D022D5C305602031DD9
:1009FE00022DC0305502031C212D5808003C031D4A
:100A0E00122D5708213C031D122D5608913C031D33
:100A1E00122D5508BF3C031C212D8B30D900061218
:100A2E008612061386132030AF006C30AD000230F4
:100A3E00AE00212D3008003A031D542D3308013A23
:100A4E00031D542D6C30F4002A30F500F601F70129
:100A5E005508F0005608F1005708F2005808F30048
:100A6E007408F0027508031C750FF1027608031C5A
:100A7E00760FF2027708031C770FF3022F08F400AB
:100A8E00F501F601F70152227008D5007108D60063
:100A9E007208D7007308D800992D3008013A031D4B
:100AAE00832D1030F4002730F500F601F7015508BC
:100ABE00F0005608F1005708F2005808F3007408C9
:100ACE00F0027508031C750FF1027608031C760FF1
:100ADE00F2027708031C770FF3022F08F400F501DA
:100AEE00F601F70152227008D5007108D60072087F
:100AFE00D7007308D800992D5508F0005608F1005C
:100B0E005708F2005808F3002F08F400F501F6011B
:100B1E00F70152227008D5007108D6007208D7006E
:100B2E007308D8001030F4002730F500F601F701F5
:100B3E005508F0005608F1005708F2005808F30067
:100B4E0095207008B1007108B2000030F200F30079
:100B5E00A030F4008630F5000130F6000030F700CA
:100B6E0052227008DB007108DC007208DD00730889
:100B7E00DE000A30F400F501F601F7019520700849
:100B8E00DB007108DC007208DD007308DE0055081A
:100B9E00F4005608F5005708F6005808F7007008DC
:100BAE00F4027108031C710FF5027208031C720F18
:100BBE00F6027308031C730FF7027408E50075083C
:100BCE00E6007608E7007708E8006630F000F101ED
:100BDE00F201F30152223108F4003208F500F60159
:100BEE00F70195207008E4003108E9003208EA00A8
:020BFE000800ED
:100C0000831203134208F0000A30F40039227008FE
:100C10008316A0007108A1000030A11BFF30A200C4
:100C2000A3000E308312B400113034020318412E99
:100C30003408353E84000008F000F101F201F301B0
:100C400083162008F00721080318210FF107220856
:100C50000318220FF20723080318230FF3070A30A3
:100C6000F400F501F601F701522270088316A00086
:100C70007108A1007208A2007308A3008312B40ACD
:100C8000142E4608F000F101F201F301831620084A
:100C9000F00721080318210FF10722080318220F7B
:100CA000F20723080318230FF3077008A000710848
:100CB000A1007208A2007308A30083124C08003A36
:100CC000031D6C2E4708003A031D6C2E8316A001ED
:100CD000A101A201A3017B2E83124C08013A031D3E
:100CE0007B2E4808003A031D7B2E8316A001A1012C
:100CF000A201A3017B2E831241082B3A031D972EDC
:100D0000831620088312D507831621080318210FA4
:100D10008312D607831622080318220F8312D707DF
:100D2000831623080318230F8312D807AD2E8316CA
:100D300020088312D50283162108031C210F831279
:100D4000D60283162208031C220F8312D7028316B1
:0C0D50002308031C230F8312D8020800A4
:100D5C0032228A110A128000840AED0A0319EE0A63
:080D6C00F003031DAE2E080088
:100D74000730831203139F00831685010330860016
:100D8400831205118510051086110516851503308B
:100D9400FB008A30FC005530FD00FD0BCF2EFC0B10
:100DA400CF2EFB0BCF2E00000000851115308316CB
:100DB400990018156A200330FB008A30FC00553076
:100DC400FD00FD0BE32EFC0BE32EFB0BE32E0000DA
:040DD4000000080013
:100DD8006400213083120313EF007A200D225A0891
:100DE8003F3A031DF92E0D22EC2E5A08493A031DED
:100DF800FF2E0D22002FEC2E5A08463A031D082F0D
:100E08000D220D220D22092FEC2EB4013408203CAE
:100E1800031C282F0D2234080C3A0319182F340804
:100E2800203A0319182F1E2F3408353E84005A081B
:100E38008000262F3408353E840030305A02F000F6
:100E480070088000B40A0A2F4C08013A031D2F2F9E
:100E5800B0010512322F05160130B0004D08053AD1
:100E680003193B2F4D08043A03193B2F3E2F01303D
:100E7800B3003F2FB30155083B3A031D502F061806
:100E8800492F2530EF007A204D2F29308312EF00AB
:100E98007A2083128515532F6400851117220800C4
:100EA800493083120313A1004630A2003B30A3004F
:100EB800A4015430A5005830A6003B30A700A80173
:100EC8005230A9005830AA003B30AB00AC01BA261A
:100ED80064001722EC26892200260F235808620690
:100EE800031D802F57086106031D802F56086006D2
:100EF800031D802F55085F060319842FE2226E2FE9
:040F08006E2F852F94
:02400E00262169
:00000001FF
